:020000040000FA
:0408000030EF05F0E0
:1008100003B23DEF04F0F2B458EF04F09EB060EF85
:1008200004F09EB268EF04F0F2A81AEF04F0F2B2FE
:100830001CEF04F00EEF05F0CD90F29207BC078E8E
:10084000078C9EA029EF04F00101463F29EF04F038
:10085000472B07AE34EF04F0CECF51F1CFCF52F19A
:1008600046C153F147C154F1CF6ACE6A0101466BCC
:10087000476B9E90CD800EEF05F00392030103EECF
:1008800000F080517F0BE92604C0EFFF802B8151DF
:10089000805D700BD8A48B8200008051815D700B4D
:1008A000D8A48B9281518019D8B407900EEF05F02F
:1008B000F2940101383F0EEF05F0392B0EEF05F0F1
:1008C0009E900101463F0EEF05F0472B0EEF05F01D
:1008D0009E92C3CF48F1C4CF49F1C28207B492EFD0
:1008E00004F03AC13EF13BC13FF13CC140F13DC192
:1008F00041F151C155F152C156F153C157F154C1A3
:1009000058F1010148514E2749514F23E86A5023BD
:100910000D2E92EF04F04FC14AF150C14BF14E6BD6
:100920004F6B506B0201002F0EEF05F03C0E006F75
:1009300001015D67A3EF04F05E67A3EF04F05F675A
:10094000A3EF04F06067A7EF04F0D7EF04F061C1F4
:1009500000F162C101F163C102F164C103F101015F
:10096000010E046F000E056F000E066F000E076F7C
:1009700083EC11F000C161F101C162F102C163F1C8
:1009800003C164F10067CCEF04F00167CCEF04F021
:100990000267CCEF04F00367D7EF04F05DC161F1AB
:1009A0005EC162F15FC163F160C164F10E80D57E0A
:1009B000D5BE32D0D6CF3AF1D7CF3BF138C13CF1DA
:1009C000E86AE8CF3DF1010147A7F2EF04F0079C88
:1009D000079E0101000E516F600E526F3D0E536F66
:1009E000080E546F01013ABF02EF05F03B6702EFBA
:1009F00005F03C6702EF05F03D6702EF05F0F28875
:100A000007EF05F0F298516B526B536B546BD76A3A
:100A1000D66A0101386B396B0EEF05F002C0E0FFBA
:100A2000005001C0D8FF1000A6B214EF05F00CC0B2
:100A3000A9FF0BC0A8FFA69EA69CA684F29E550EF9
:100A4000A76EAA0EA76EA682F28EA694A6B226EF75
:100A500005F01200A96EA69EA69CA680A8501200C2
:100A6000076A0E6A0F010E0EC16E860EC06E030E6F
:100A7000C26E0F01896A110E926E080E8A6EF10E17
:100A8000936E8B6A800E946EF18E0D6A4E6B4F6B77
:100A9000506B4A6B4B6B0F01280ED56EF28AB00E6D
:100AA000CD6E9D800101516B526B536B546B556B36
:100AB000566B576B586B596B5A6B5B6B5C6B079C37
:100AC000079E760ECA6E9D8202013C0E006FCC6AB4
:100AD000160E2AEC05F0E8CF00F1170E2AEC05F00F
:100AE000E8CF01F1180E2AEC05F0E8CF02F1190E5B
:100AF0002AEC05F0E8CF03F1010103AF9AEF05F00E
:100B00007AEC12F0160E0C6E00C10BF014EC05F02E
:100B1000170E0C6E01C10BF014EC05F0180E0C6EE4
:100B200002C10BF014EC05F0190E0C6E03C10BF0B2
:100B300014EC05F000C15DF101C15EF102C15FF18D
:100B400003C160F100C161F101C162F102C163F151
:100B500003C164F11A0E2AEC05F0E8CF00F11B0E78
:100B60002AEC05F0E8CF01F11C0E2AEC05F0E8CFE5
:100B700002F11D0E2AEC05F0E8CF03F1010103AFED
:100B8000F0EF05F07AEC12F01A0E0C6E00C10BF0CB
:100B900014EC05F01B0E0C6E01C10BF014EC05F00B
:100BA0001C0E0C6E02C10BF014EC05F01D0E0C6E49
:100BB00003C10BF014EC05F01A0E2AEC05F0E8CF97
:100BC00000F11B0E2AEC05F0E8CF01F11C0E2AEC17
:100BD00005F0E8CF02F11D0E2AEC05F0E8CF03F195
:100BE00000C165F101C166F102C167F103C168F19D
:100BF000240EAC6E0401806B816B0F01900EAB6E06
:100C00000F019D8A0301806B816BA26B8B92079011
:100C10000001F28EF28C07B08EEF0FF00EB08AEF6B
:100C20000AF00301805181197F0BD8B48EEF0FF0C9
:100C300013EE00F081517F0BE126812BE7CFE8FF17
:100C4000E00BD8B48EEF0FF023EE82F0A2511F0B11
:100C5000D926E7CFDFFFA22BDF50780AD8A48EEF8A
:100C60000FF0078061C100F162C101F163C102F1BF
:100C700064C103F10101040E046F000E056F000E44
:100C8000066F000E076F83EC11F000AF51EF06F016
:100C90000101030E616F000E626F000E636F000EA4
:100CA000646F03018251720AD8B48AEF0AF082514C
:100CB000630AD8B44EEF0CF08251690AD8B45FEFE2
:100CC00008F082517A0AD8B472EF09F08251490AC9
:100CD000D8B476EF07F08251500AD8B494EF06F0FA
:100CE0008251700AD8B4D7EF06F08251540AD8B4B2
:100CF00002EF07F08251740AD8B448EF07F083EF8F
:100D00000CF0040114EE00F080517F0BE12682C448
:100D1000E7FF802B12000D0E826F81EC06F00A0EA9
:100D2000826F81EC06F0120083C31EF184C31FF1B1
:100D300085C320F186C321F187C322F188C323F143
:100D400089C324F18AC325F18BC326F18CC327F113
:100D50000101C7EC12F03FEC12F0160E0C6E00C150
:100D60000BF014EC05F0170E0C6E01C10BF014EC37
:100D700005F0180E0C6E02C10BF014EC05F0190E04
:100D80000C6E03C10BF014EC05F000C15DF101C164
:100D90005EF102C15FF103C160F100C161F101C107
:100DA00062F102C163F103C164F176EF07F083C31E
:100DB0001EF184C31FF185C320F186C321F187C3CF
:100DC00022F188C323F189C324F18AC325F18BC39F
:100DD00026F18CC327F10101C7EC12F03FEC12F0B1
:100DE00000C15DF101C15EF102C15FF103C160F1BB
:100DF00000C161F101C162F102C163F103C164F19B
:100E000076EF07F083C31EF184C31FF185C320F181
:100E100086C321F187C322F188C323F189C324F15A
:100E20008AC325F18CC326F18DC327F10101C7ECDC
:100E300012F03FEC12F00101000E046F000E056F7E
:100E4000010E066F000E076F92EC11F01A0E0C6E79
:100E500000C10BF014EC05F01B0E0C6E01C10BF081
:100E600014EC05F01C0E0C6E02C10BF014EC05F036
:100E70001D0E0C6E03C10BF014EC05F000C165F102
:100E800001C166F102C167F103C168F176EF07F0B5
:100E900083C31EF184C31FF185C320F186C321F1F2
:100EA00087C322F188C323F189C324F18AC325F1C2
:100EB0008CC326F18DC327F10101C7EC12F03FEC82
:100EC00012F00101000E046F000E056F010E066F97
:100ED000000E076F92EC11F000C165F101C166F1DF
:100EE00002C167F103C168F176EF07F0160E2AEC34
:100EF00005F0E8CF00F1170E2AEC05F0E8CF01F17C
:100F0000180E2AEC05F0E8CF02F1190E2AEC05F0D4
:100F1000E8CF03F11DEC12F01EC182F40401300E83
:100F2000822781EC06F01FC182F40401300E822773
:100F300081EC06F020C182F40401300E822781EC9E
:100F400006F021C182F40401300E822781EC06F004
:100F500022C182F40401300E822781EC06F023C105
:100F600082F40401300E822781EC06F024C182F461
:100F70000401300E822781EC06F025C182F40401C1
:100F8000300E822781EC06F026C182F40401300E77
:100F9000822781EC06F027C182F40401300E8227FB
:100FA00081EC06F00401730E826F81EC06F00401FF
:100FB0002C0E826F81EC06F05DC100F15EC101F183
:100FC0005FC102F160C103F11DEC12F01EC182F499
:100FD0000401300E822781EC06F01FC182F4040167
:100FE000300E822781EC06F020C182F40401300E1D
:100FF000822781EC06F021C182F40401300E8227A1
:1010000081EC06F022C182F40401300E822781ECCB
:1010100006F023C182F40401300E822781EC06F031
:1010200024C182F40401300E822781EC06F025C130
:1010300082F40401300E822781EC06F026C182F48E
:101040000401300E822781EC06F027C182F40401EE
:10105000300E822781EC06F00401730E826F81EC62
:1010600006F004012C0E826F81EC06F01A0E2AECB9
:1010700005F0E8CF00F11B0E2AEC05F0E8CF01F1F6
:101080001C0E2AEC05F0E8CF02F11D0E2AEC05F04B
:10109000E8CF03F19DEC0CF004012C0E826F81EC83
:1010A00006F065C100F166C101F167C102F168C1D6
:1010B00003F19DEC0CF08BEC06F083EF0CF00401D7
:1010C000690E826F81EC06F004012C0E826F81ECB8
:1010D00006F00101030E006F000E016F000E026F9B
:1010E000000E036F1DEC12F020C182F40401300EDB
:1010F000822781EC06F021C182F40401300E8227A0
:1011000081EC06F022C182F40401300E822781ECCA
:1011100006F023C182F40401300E822781EC06F030
:1011200024C182F40401300E822781EC06F025C12F
:1011300082F40401300E822781EC06F026C182F48D
:101140000401300E822781EC06F027C182F40401ED
:10115000300E822781EC06F004012C0E826F81ECA8
:1011600006F00101030E006F000E016F000E026F0A
:10117000000E036F1DEC12F020C182F40401300E4A
:10118000822781EC06F021C182F40401300E82270F
:1011900081EC06F022C182F40401300E822781EC3A
:1011A00006F023C182F40401300E822781EC06F0A0
:1011B00024C182F40401300E822781EC06F025C19F
:1011C00082F40401300E822781EC06F026C182F4FD
:1011D0000401300E822781EC06F027C182F404015D
:1011E000300E822781EC06F004012C0E826F81EC18
:1011F00006F001010D0E006F000E016F000E026F70
:10120000000E036F1DEC12F020C182F40401300EB9
:10121000822781EC06F021C182F40401300E82277E
:1012200081EC06F022C182F40401300E822781ECA9
:1012300006F023C182F40401300E822781EC06F00F
:1012400024C182F40401300E822781EC06F025C10E
:1012500082F40401300E822781EC06F026C182F46C
:101260000401300E822781EC06F027C182F40401CC
:10127000300E822781EC06F004012C0E826F81EC87
:1012800006F0200EF86EF76AF66A04010900F5CF41
:1012900082F481EC06F00900F5CF82F481EC06F0CF
:1012A0000900F5CF82F481EC06F00900F5CF82F455
:1012B00081EC06F00900F5CF82F481EC06F009001C
:1012C000F5CF82F481EC06F00900F5CF82F481ECD1
:1012D00006F00900F5CF82F481EC06F08BEC06F005
:1012E00083EF0CF08351630AD8A483EF0CF0845190
:1012F000610AD8A483EF0CF085516C0AD8A483EF5F
:101300000CF08651410A42E08651440A1BE08651A6
:10131000420AD8B4D9EF09F08651350AD8B40CEF97
:101320000EF08651360AD8B460EF0EF08651370AB7
:10133000D8B4C8EF0EF08651380AD8B426EF0FF0B3
:1013400083EF0CF00798079A04017A0E826F81EC04
:1013500006F00401780E826F81EC06F00401640E41
:10136000826F81EC06F081A8BDEF09F00401550EF3
:10137000826F81EC06F0C2EF09F004014C0E826F1F
:1013800081EC06F08BEC06F083EF0CF00788079AEF
:1013900004017A0E826F81EC06F00401410E826F27
:1013A00081EC06F00401610E826F81EC06F0B3EF70
:1013B00009F00798078A04017A0E826F81EC06F023
:1013C0000401420E826F81EC06F00401610E826F0F
:1013D00081EC06F0B3EF09F00101620E046F010E1B
:1013E000056F000E066F000E076F59C100F15AC15C
:1013F00001F15BC102F15CC103F183EC11F003BFA9
:1014000049EF0AF00E0E2AEC05F0E8CF0CF10F0EB2
:101410002AEC05F0E8CF0DF1100E2AEC05F0E8CF2C
:101420000EF1110E2AEC05F0E8CF0FF1CCEC10F024
:1014300059C104F15AC105F15BC106F15CC107F164
:1014400083EC11F0078290EC10F0CCEC10F00792D6
:1014500090EC10F059C100F15AC101F15BC102F1E9
:101460005CC103F1079290EC10F0CC0E046FE00E1B
:10147000056F870E066F050E076F83EC11F000C134
:101480000CF101C10DF102C10EF103C10FF181EFA9
:101490000AF00101800E006F1A0E016F060E026F36
:1014A000000E036F42C104F143C105F144C106F1CE
:1014B00045C107F183EC11F003AF62EF0AF07AEC5B
:1014C00012F012000E0E2AEC05F0E8CF0CF10F0E10
:1014D0002AEC05F0E8CF0DF1100E2AEC05F0E8CF6C
:1014E0000EF1110E2AEC05F0E8CF0FF142C100F128
:1014F00043C101F144C102F145C103F1078290ECFF
:1015000010F00CC100F10DC101F10EC102F10FC1CB
:1015100003F11200078455C159F156C15AF157C160
:101520005BF158C15CF13EC142F13FC143F140C1A2
:1015300044F141C145F14AC14CF14BC14DF1079411
:101540000EA0C2EF0AF00E9001016567AFEF0AF03E
:101550006667AFEF0AF06767AFEF0AF06867B3EF4F
:101560000AF0C2EF0AF0ECEC09F065C104F166C1C3
:1015700005F167C106F168C107F183EC11F003BF03
:1015800083EF0CF0ECEC09F00101000E046F000E8B
:10159000056F010E066F000E076FB1EC11F004012C
:1015A000720E826F81EC06F004012C0E826F81ECCA
:1015B00006F01DEC12F01D67E3EF0AF00401200EA7
:1015C000826FE6EF0AF004012D0E826F81EC06F0C7
:1015D00024C182F40401300E822781EC06F025C17B
:1015E00082F40401300E822781EC06F004012E0EF5
:1015F000826F81EC06F026C182F40401300E82274E
:1016000081EC06F027C182F40401300E822781ECC0
:1016100006F004016D0E826F81EC06F004012C0EC1
:10162000826F81EC06F042C100F143C101F144C177
:1016300002F145C103F101011DEC12F01EC182F45B
:101640000401300E822781EC06F01FC182F40401F0
:10165000300E822781EC06F020C182F40401300EA6
:10166000822781EC06F021C182F40401300E82272A
:1016700081EC06F022C182F40401300E822781EC55
:1016800006F023C182F40401300E822781EC06F0BB
:1016900024C182F40401300E822781EC06F025C1BA
:1016A00082F40401300E822781EC06F026C182F418
:1016B0000401300E822781EC06F027C182F4040178
:1016C000300E822781EC06F00401480E826F81EC17
:1016D00006F004017A0E826F81EC06F004012C0EF4
:1016E000826F81EC06F059C100F15AC101F15BC172
:1016F00002F15CC103F101011DEC12F01EC182F484
:101700000401300E822781EC06F01FC182F404012F
:10171000300E822781EC06F020C182F40401300EE5
:10172000822781EC06F021C182F40401300E822769
:1017300081EC06F022C182F40401300E822781EC94
:1017400006F023C182F40401300E822781EC06F0FA
:1017500024C182F40401300E822781EC06F025C1F9
:1017600082F40401300E822781EC06F026C182F457
:101770000401300E822781EC06F027C182F40401B7
:10178000300E822781EC06F00401630E826F81EC3B
:1017900006F004012C0E826F81EC06F059C100F1B5
:1017A0005AC101F15BC102F15CC103F101010A0EF2
:1017B000046F000E056F000E066F000E076F92ECAF
:1017C00011F0000E046F120E056F000E066F000E72
:1017D000076FB1EC11F01DEC12F01EC182F4040190
:1017E000300E822781EC06F01FC182F40401300E16
:1017F000822781EC06F020C182F40401300E82279A
:1018000081EC06F021C182F40401300E822781ECC4
:1018100006F022C182F40401300E822781EC06F02A
:1018200023C182F40401300E822781EC06F024C12A
:1018300082F40401300E822781EC06F004012E0EA2
:10184000826F81EC06F025C182F40401300E8227FC
:1018500081EC06F026C182F40401300E822781EC6F
:1018600006F027C182F40401300E822781EC06F0D5
:101870000401730E826F81EC06F004012C0E826F5E
:1018800081EC06F07AEC12F04CC100F14DC101F18F
:10189000ACEC0DF08BEC06F083EF0CF00401630E62
:1018A000826F81EC06F004012C0E826F81EC06F051
:1018B00088EC0CF004012C0E826F81EC06F0FBEC3E
:1018C0000CF004012C0E826F81EC06F077EC0DF029
:1018D00004012C0E826F81EC06F00101F80E006FFE
:1018E000CD0E016F660E026F030E036F9DEC0CF0C0
:1018F00004012C0E826F81EC06F08DEC0DF08BEC68
:1019000006F083EF0CF00301A26B07908EEF0FF04F
:10191000D8900E0E2AEC05F0E8CF00F10F0E2AEC5D
:1019200005F0E8CF01F1100E2AEC05F0E8CF02F146
:10193000110E2AEC05F0E8CF03F10101000E046F4F
:10194000000E056F010E066F000E076FB1EC11F06F
:101950001DEC12F01EC182F40401300E822781ECCE
:1019600006F01FC182F40401300E822781EC06F0DC
:1019700020C182F40401300E822781EC06F021C1DF
:1019800082F40401300E822781EC06F022C182F439
:101990000401300E822781EC06F023C182F4040199
:1019A000300E822781EC06F024C182F40401300E4F
:1019B000822781EC06F025C182F40401300E8227D3
:1019C00081EC06F004012E0E826F81EC06F026C138
:1019D00082F40401300E822781EC06F027C182F4E4
:1019E0000401300E822781EC06F004016D0E826F37
:1019F00081EC06F01200120E2AEC05F0E8CF00F19F
:101A0000130E2AEC05F0E8CF01F1140E2AEC05F0D4
:101A1000E8CF02F1150E2AEC05F0E8CF03F1010141
:101A20000A0E046F000E056F000E066F000E076FA2
:101A300092EC11F0000E046F120E056F000E066F8F
:101A4000000E076FB1EC11F01DEC12F01EC182F414
:101A50000401300E822781EC06F01FC182F40401DC
:101A6000300E822781EC06F020C182F40401300E92
:101A7000822781EC06F021C182F40401300E822716
:101A800081EC06F022C182F40401300E822781EC41
:101A900006F023C182F40401300E822781EC06F0A7
:101AA00024C182F40401300E822781EC06F0040187
:101AB0002E0E826F81EC06F025C182F40401300EF7
:101AC000822781EC06F026C182F40401300E8227C1
:101AD00081EC06F027C182F40401300E822781ECEC
:101AE00006F00401730E826F81EC06F012000A0EFC
:101AF0002AEC05F0E8CF00F10B0E2AEC05F0E8CF58
:101B000001F10C0E2AEC05F0E8CF02F10D0E2AECE3
:101B100005F0E8CF03F1ACEF0DF0060E2AEC05F06E
:101B2000E8CF00F1070E2AEC05F0E8CF01F1080E2E
:101B30002AEC05F0E8CF02F1090E2AEC05F0E8CF17
:101B400003F1ACEF0DF001017AEC12F007844AC109
:101B500000F14BC101F107940101E80E046F800E02
:101B6000056F000E066F000E076F92EC11F0000E6D
:101B7000046F040E056F000E066F000E076FB1ECC8
:101B800011F0880E046F130E056F000E066F000E25
:101B9000076F83EC11F00A0E046F000E056F000E44
:101BA000066F000E076FB1EC11F01DEC12F0010191
:101BB0001D67E0EF0DF00401200E826FE3EF0DF0E2
:101BC00004012D0E826F81EC06F024C182F4040121
:101BD000300E822781EC06F025C182F40401300E1C
:101BE000822781EC06F026C182F40401300E8227A0
:101BF00081EC06F004012E0E826F81EC06F027C105
:101C000082F40401300E822781EC06F00401430EB9
:101C1000826F81EC06F0120087C31EF188C31FF1AA
:101C200089C320F18AC321F18BC322F18CC323F134
:101C30008DC324F18EC325F190C326F191C327F102
:101C40000101C7EC12F03FEC12F00101000E046F2D
:101C5000000E056F010E066F000E076F92EC11F07B
:101C60000E0E0C6E00C10BF014EC05F00F0E0C6E96
:101C700001C10BF014EC05F0100E0C6E02C10BF05C
:101C800014EC05F0110E0C6E03C10BF014EC05F012
:101C900004017A0E826F81EC06F004012C0E826F33
:101CA00081EC06F00401350E826F81EC06F0040130
:101CB0002C0E826F81EC06F088EC0CF0C2EF09F07C
:101CC00087C31EF188C31FF189C320F18AC321F1A4
:101CD0008BC322F18CC323F18DC324F18EC325F174
:101CE00090C326F191C327F10101C7EC12F03FEC3C
:101CF00012F0880E046F130E056F000E066F000EB3
:101D0000076F87EC11F0000E046F040E056F000ED4
:101D1000066F000E076F92EC11F00101E80E046FE0
:101D2000800E056F000E066F000E076FB1EC11F00C
:101D30000A0E0C6E00C10BF014EC05F00B0E0C6ECD
:101D400001C10BF014EC05F00C0E0C6E02C10BF08F
:101D500014EC05F00D0E0C6E03C10BF014EC05F045
:101D600004017A0E826F81EC06F004012C0E826F62
:101D700081EC06F00401360E826F81EC06F004015E
:101D80002C0E826F81EC06F077EC0DF0C2EF09F0BB
:101D900087C31EF188C31FF189C320F18AC321F1D3
:101DA0008BC322F18CC323F18DC324F18FC325F1A2
:101DB00090C326F191C327F10101C7EC12F03FEC6B
:101DC00012F0000E046F120E056F000E066F000E6B
:101DD000076F92EC11F001010A0E046F000E056FFF
:101DE000000E066F000E076FB1EC11F0120E0C6EB4
:101DF00000C10BF014EC05F0130E0C6E01C10BF0DA
:101E000014EC05F0140E0C6E02C10BF014EC05F08E
:101E1000150E0C6E03C10BF014EC05F004017A0EE4
:101E2000826F81EC06F004012C0E826F81EC06F0CB
:101E30000401370E826F81EC06F004012C0E826FD4
:101E400081EC06F0FBEC0CF0C2EF09F087C31EF149
:101E500088C31FF189C320F18AC321F18BC322F10A
:101E60008CC323F18DC324F18EC325F190C326F1D9
:101E700091C327F10101C7EC12F03FEC12F0880E7C
:101E8000046F130E056F000E066F000E076F87ECD0
:101E900011F0000E046F040E056F000E066F000EA9
:101EA000076F92EC11F00101E80E046F800E056FD0
:101EB000000E066F000E076FB1EC11F0060E0C6EEF
:101EC00000C10BF014EC05F0070E0C6E01C10BF015
:101ED00014EC05F0080E0C6E02C10BF014EC05F0CA
:101EE000090E0C6E03C10BF014EC05F004017A0E20
:101EF000826F81EC06F004012C0E826F81EC06F0FB
:101F00000401380E826F81EC06F004012C0E826F02
:101F100081EC06F08DEC0DF0C2EF09F081A84CEFDA
:101F200010F007A805EF10F00101800E006F1A0EE7
:101F3000016F060E026F000E036F3EC104F13FC138
:101F400005F140C106F141C107F183EC11F003BF77
:101F50004CEF10F08AEC10F03EC100F13FC101F1EE
:101F600040C102F141C103F1078290EC10F00CC1B5
:101F700004F10DC105F10EC106F10FC107F1F80E14
:101F8000006FCD0E016F660E026F030E036F83ECC0
:101F900011F00E0E0C6E00C10BF014EC05F00F0EDC
:101FA0000C6E01C10BF014EC05F0100E0C6E02C1AA
:101FB0000BF014EC05F0110E0C6E03C10BF014ECD9
:101FC00005F0078401017AEC12F04AC100F14BC11F
:101FD00001F107940A0E0C6E00C10BF014EC05F031
:101FE0000B0E0C6E01C10BF014EC05F00C0E0C6E18
:101FF00002C10BF014EC05F00D0E0C6E03C10BF0DA
:1020000014EC05F007984CEF10F007AA4CEF10F015
:10201000078401017AEC12F04AC100F14BC101F1D1
:102020000794060E0C6E00C10BF014EC05F0070EC1
:102030000C6E01C10BF014EC05F0080E0C6E02C121
:102040000BF014EC05F0090E0C6E03C10BF014EC50
:1020500005F0078455C100F156C101F157C102F1E5
:1020600058C103F10794120E0C6E00C10BF014EC72
:1020700005F0130E0C6E01C10BF014EC05F0140EFC
:102080000C6E02C10BF014EC05F0150E0C6E03C1C2
:102090000BF014EC05F0079A0401805181197F0BB5
:1020A0000BE09EA809D014EE00F081517F0BE126D1
:1020B000E750812B0F01AD6E0BEF06F00CC100F164
:1020C0000DC101F10EC102F10FC103F1000E046F49
:1020D000000E056F010E066F000E076FB1EC11F0D8
:1020E0001DA189EF10F01451D8B489EF10F00CC184
:1020F00000F10DC101F10EC102F10FC103F1000E9B
:10210000046F000E056F0A0E066F000E076FB1EC2C
:1021100011F0120001010C6B0D6B0E6B0F6B1200B6
:102120000101005305E1015303E1025301E1002BDA
:1021300053EC11F07AEC12F02C51006F2D51016F1D
:10214000420E046F4B0E056F000E066F000E076FF8
:1021500092EC11F000C104F101C105F102C106F1D8
:1021600003C107F10CC100F10DC101F10EC102F173
:102170000FC103F107B2C1EF10F087EC11F0C3EF0C
:1021800010F083EC11F000C10CF101C10DF102C19E
:102190000EF103C10FF112007AEC12F04CC100F104
:1021A0004DC101F1060E2AEC05F0E8CF04F1070E4F
:1021B0002AEC05F0E8CF05F1080E2AEC05F0E8CF8F
:1021C00006F1090E2AEC05F0E8CF07F183EC11F0D7
:1021D00000C118F101C119F102C11AF103C11BF1CB
:1021E000290E046F000E056F000E066F000E076FBC
:1021F00092EC11F0EE0E046F430E056F000E066FA9
:10220000000E076F87EC11F018C104F119C105F138
:102210001AC106F11BC107F192EC11F000C110F1D7
:1022200001C111F102C112F103C113F1120E2AEC26
:1022300005F0E8CF04F1130E2AEC05F0E8CF05F124
:10224000140E2AEC05F0E8CF06F1150E2AEC05F085
:10225000E8CF07F10D0E006F000E016F000E026F48
:10226000000E036F92EC11F0180E046F000E056F54
:10227000000E066F000E076FB1EC11F010C104F1F3
:1022800011C105F112C106F113C107F187EC11F07C
:102290006A0E046F2A0E056F000E066F000E076FA0
:1022A00083EC11F01200BF0EFA6E200E2D6F2C6B16
:1022B000D8900037013702370337D8B064EF11F0F8
:1022C0002D2F59EF11F02C072D070353D8B412000E
:1022D0000331070B8009326F03390F0B010F2C6F8D
:1022E00080EC5FF0336F2C0580EC5FF0335D335F83
:1022F0002C6B3233D8B02C272C3332A979EF11F064
:1023000033512C2712009FEC12F0D8B01200035169
:102310000719286F62EC12F0D8900751031928AF03
:10232000800F1200286B86EC12F0D8A09CEC12F003
:10233000D8B0120071EC12F07AEC12F01F0E296F77
:10234000B2EC12F00B35D8B062EC12F0D8A0033525
:10235000D8B01200292FA0EF11F028B189EC12F0AB
:102360001200286B04510511061107110008D8A0AE
:1023700086EC12F0D8A09CEC12F0D8B01200086BDA
:10238000096B0A6B0B6BB2EC12F01F0E296FB2ECEB
:1023900012F007510B5DD8A4DAEF11F006510A5D77
:1023A000D8A4DAEF11F00551095DD8A4DAEF11F0E5
:1023B0000451085DD8A0EDEF11F00451085F0551FC
:1023C000D8A0053D095F0651D8A0063D0A5F075118
:1023D000D8A0073D0B5FD8900081292FC7EF11F0DF
:1023E00028B189EC12F0286B86EC12F0D890B6EC8C
:1023F00012F007510B5DD8A40AEF12F006510A5DE6
:10240000D8A40AEF12F00551095DD8A40AEF12F022
:102410000451085DD8A019EF12F0003F19EF12F037
:10242000013F19EF12F0023F19EF12F0032BD8B45D
:10243000120028B189EC12F012000101286B86EC21
:1024400012F0D8B01200BBEC12F0200E296F00374A
:1024500001370237033711EE27F00A0E2A6FE736ED
:102460000A0EE75CD8B0E76EE5522A2F2FEF12F084
:10247000292F27EF12F028B11D81D89012000101F9
:102480000A0E286F200E296F11EE1DF028512A6FB9
:102490000A0ED890E652D8B0E726E7322A2F4AEF44
:1024A00012F00333023301330033292F44EF12F0CB
:1024B000E750FF0FD8A00335D8B012001DB189EC4A
:1024C00012F01200045100270551D8B0053D012734
:1024D0000651D8B0063D02270751D8B0073D032763
:1024E00012000051086F0151096F02510A6F035128
:1024F0000B6F12000101006B016B026B036B12008A
:102500000101046B056B066B076B12000335D8A045
:1025100012000351800B001F011F021F031F003F09
:1025200099EF12F0013F99EF12F0023F99EF12F08C
:10253000032B282B032512000735D8A012000751C2
:10254000800B041F051F061F071F043FAFEF12F08B
:10255000053FAFEF12F0063FAFEF12F0072B282B2D
:1025600007251200003701370237033708370937CC
:102570000A370B3712001D6B1E6B1F6B206B216B14
:10258000226B236B246B256B266B276B12001E516D
:102590000F0B1E6F1F510F0B1F6F20510F0B206F62
:1025A00021510F0B216F22510F0B226F23510F0B63
:1025B000236F24510F0B246F25510F0B256F2651CC
:0C25C0000F0B266F27510F0B276F120026
:10BF0000E844F926000C160C2B0C3F0C520C640C68
:10BF1000760C860C960CA50CB30CC10CCF0CDC0C6B
:06BF2000E80CF40C000C1B
:00000001FF
